:020000040800F2
:10000000984500204D01000859190008C511000845
:1000100055190008C3020008B92C000800000000B0
:10002000000000000000000000000000FF1B0008AE
:10003000430B00080000000063010008691D000870
:1000400067010008670100086701000867010008F0
:1000500067010008670100086701000867010008E0
:1000600067010008670100086701000867010008D0
:100070008D090008670100088F0900086701000862
:1000800067010008670100086701000867010008B0
:1000900067010008670100086701000867010008A0
:1000A0006701000867010008670100086701000890
:1000B0006701000867010008670100086701000880
:1000C0006701000867010008670100086701000870
:1000D000670100084D270008552700085D27000824
:1000E0006701000867010008670100086701000850
:1000F0006701000867010008670100086701000840
:10010000670100086701000867010008670100082F
:10011000670100086701000867010008670100081F
:10012000670100086701000867010008670100080F
:10013000DFF80CD000F094F8004800479D37000825
:100140009845002080F308887047000006488047E3
:1001500006480047FEE7FEE7FEE7FEE7FEE7FEE7AC
:10016000FEE7FEE7FEE7FEE7911D0008310100080B
:1001700040EA01039B0703D009E008C9121F08C029
:10018000042AFAD203E011F8013B00F8013B521EA9
:10019000F9D27047D2B201E000F8012B491EFBD220
:1001A00070470022F6E710B513460A460446194682
:1001B000FFF7F0FF204610BD421E12F8013F002B52
:1001C000FBD111F8013B02F8013B002BF9D170473C
:1001D00010B5002200E0521C835C8C5CA34201D16C
:1001E000002BF8D1D8B2E1B2401A10BD034611F885
:1001F000012B00F8012B002AF9D1184670472DE990
:10020000F05F0546002092469B468846064681469A
:1002100040241BE0284641464746224600F041F86C
:1002200053465A46C01A914110D3114618462246E9
:1002300000F028F82D1A67EB01084F4622460120EE
:10024000002100F01FF817EB00094E41201EA4F119
:100250000104DFDC484631462A464346BDE8F09FAC
:10026000064C074D06E0E06840F0010394E8070003
:1002700098471034AC42F6D3FFF75EFFF43E000817
:10028000143F0008202A04DB203A00FA02F1002083
:1002900070479140C2F1200320FA03F319439040C4
:1002A0007047202A04DB203A21FA02F0002170472F
:1002B00021FA02F3D040C2F12002914008431946CE
:1002C000704700BFFEE700002DE9F05F05460E46CF
:1002D00006EB460000EBC60105F1080000EB8100CB
:1002E000D0F8249006EB460000EBC60105F10800AB
:1002F00000EB8100D0F828B00027B846BA4624E0C9
:10030000A9EB080011490988884202D30F480488E4
:1003100006E0A9EB080084B20AF1010000F0FF0A30
:100320000B4A5A44D1190B4A5068224603F0EAFAA4
:10033000084821464268384600F0E4F8BAF1000F58
:1003400001D0BDE8F09FA0442744D9E7A4000020D5
:1003500000102000640000202DE9F04F85B0074612
:100360004FF480554FF000090DE009EB490000EB18
:10037000C90107F1080000EB8100406A054409F15A
:10038000010000F0FF0978684845EED800260024F7
:10039000A2463BE0281B20490988884203D31E4817
:1003A000B0F8008006E0281B1FFA80F80AF101006F
:1003B00000F0FF0A19494246486819493144491C6E
:1003C00003F0A0FA154942464868314603F00EFB97
:1003D0004644444464206043B0FBF5F000F0FF0B5A
:1003E000019858450ED0CDF804B064206043B0FBAE
:1003F000F5F002460BA1009002A802F021FD02A830
:1004000001F0F0F8BAF1000F00D000E0C2E700BF41
:1004100005B0BDE8F08F0000A400002064000020BB
:10042000FFFF1F00436F7079202564200D0A000034
:1004300070B5ADF5786D28480078022802D00DF52A
:10044000786D70BD6E464FF478624FF400113046FF
:1004500003F058FA2149009888423BD1002220A19C
:10046000684600F0BCFD0546681C00D1E7E7E9B22C
:100470006846FFF729FF6846FFF76EFF002412E089
:1004800004EB440000EBC40102A800EB8100806A89
:1004900000F5805004EB440101EBC40202A901EB1A
:1004A00082018862641C0198A042E9D84FF4786206
:1004B0000021304603F09AFA0B4800900422D10440
:1004C000304603F093FA0948009004220021304698
:1004D00003F08CFA00BFB2E764000020A9CBED9FC7
:1004E000485331350D0A000087D52F75F8DEBC8AD8
:1004F00002200249087002484860704764000020EA
:100500000A0100202DE9F04104460D461646002759
:1005100014F0010F02D00020BDE8F081AAB2044916
:1005200009680819314602F045FC0120F4E7000093
:10053000A00000202DE9F04104460D461646334642
:100540002A462146044801F0B9F9074639460248CF
:1005500002F09CFBBDE8F081AE21002010B50448FC
:1005600001F0DAF904462146014802F08FFB10BD84
:10057000AE2100202DE9F04FB5B00646B246DAF8BC
:100580000000E049884204D04FF0FF3035B0BDE8AC
:10059000F08F9AF80400952802D06FF00100F5E77B
:1005A0009AF805B0BAF818000290BBF1030F7CD19D
:1005B0000298A0F57061823902D06FF00300E5E780
:1005C0003546B5F89A9F4FF4786205F11A0100207C
:1005D00002F088FF8046C84502D06FF00400D5E7DE
:1005E000D5F81E0008B90020D0E705F11A0000F088
:1005F00013FCC5490880D5F81E000988884209D82F
:10060000D5F81E00C1494860C148086000F0F8FBF9
:100610000020BBE7D5F81E00BC494860D5F81E3065
:10062000DFF8E4C2BCF800C0A3EB0C034FF02C0CC5
:1006300003FB0CF2B44B1B8803EB430C0CEBC30C19
:1006400005F1220303EB8C01AF4B1B8803EB430C3A
:100650000CEBC30CAD4B083303EB8C00FFF788FDAC
:100660000020AC490860A9484268ABA103A802F089
:10067000E7FB03A800F0B6FFA348008800EB4001A9
:1006800001EBC001A148083000EB8100406A0090F6
:100690009D48008800EB400101EBC0019B480830F9
:1006A00000EB81039848028800E010E09FA103A8B6
:1006B00002F0C6FB03A800F095FF4FF48052954866
:1006C000016891480088FFF735FF01205EE7BBF124
:1006D000040F75D13446D4F83E10B4F8460000EB50
:1006E000400202EBC0028948083000EB8200406AF9
:1006F00081420AD1A06C87490968884205D1B4F8C3
:1007000046008149098888420DD08EA000F06AFF1A
:100710004FF480527F4801687B480088FFF70AFF4A
:100720006FF0050032E7E76CBF1E3A4604F1500156
:10073000002002F0D7FE814604F15000791C405C95
:100740004FEA002804F15000C05D40441FFA80F8D1
:10075000C8450DD084A000F045FF4FF480526D488D
:10076000016869480088FFF7E5FE6FF007000DE7B4
:10077000BAB26548008800EB400303EBC00363484E
:10078000083000EB8300806A624B1B68C11804F1DB
:10079000500003F02BF95F4800683918D4F83E0088
:1007A00081427DD359484068401E57490988884294
:1007B00007D157485549086000F022FB0020E5E6C4
:1007C0009DE05148008800F093FA50BB0020514949
:1007D00008604D48008800EB400101EBC0014B4828
:1007E000083000EB8100406A00904748008800EB29
:1007F000400101EBC0014548083000EB810342484D
:1008000002884AA103A802F01BFB03A800F0EAFE3D
:100810004FF480523F4801683B480088FFF78AFE4A
:100820006BE039480088401C37490880084600883A
:10083000401E00EB400101EBC0013448083000EBE2
:100840008100816A30480088401E00EB400202EBC4
:10085000C0022E48083000EB8200406A01442A485A
:10086000008800EB400202EBC0022848083000EB91
:10087000820081620020274908602348008800EB3D
:10088000400101EBC0012148083000EB8100406AC3
:1008900000901D48008800EB400101EBC00100E022
:1008A00015E01A48083000EB8103174802881FA1A1
:1008B00003A802F0C5FA03A800F094FE4FF480529A
:1008C0001448016810480088FFF734FE15E011480D
:1008D000006838440F490860084629A1026803A847
:1008E00002F0AEFA03A800F07DFE4FF480520948F2
:1008F000016805480088FFF71DFE022046E600BF9C
:1009000044E6000050435441D00000201222002051
:10091000F8DEBC8AD40000205246696C6520436F23
:10092000756E743D256C750D0A0000005246696CA9
:10093000655B25645D3A257320206C656E3D256CF2
:10094000750D0A0046696C65204C656E67746820F9
:100950006F72204F6666736574206572726F7221C4
:100960005265444F210D0A00436865636B20435272
:1009700043206572726F72215265444F210D0A0047
:100980006F66667365743D25640D0A007047704795
:1009900021B1026842F00102026004E002684FF6F1
:1009A000FE731A400260704701684FF6FE721140F4
:1009B00001600021016041608160C1604B49884253
:1009C00008D14A490839496841F00F01474A083AB5
:1009D00051608AE045491431884208D143490839B9
:1009E000496841F0F001414A083A51607DE03F49D1
:1009F0002831884208D13D490839496841F470617D
:100A00003A4A083A516070E038493C31884208D18E
:100A100036490839496841F47041344A083A51600E
:100A200063E032495031884208D130490839496879
:100A300041F470212D4A083A516056E02B49643147
:100A4000884208D129490839496841F47001274A88
:100A5000083A516049E025497831884208D1234954
:100A60000839496841F07061204A083A51603CE019
:100A70001F49884206D1011F096841F00F01021F7A
:100A8000116032E01A491431884208D11849091F0F
:100A9000096841F0F001164A121F116025E014495F
:100AA0002831884208D11249091F096841F4706150
:100AB0000F4A121F116018E00D493C31884208D1DD
:100AC0000B49091F096841F47041094A121F11605E
:100AD0000BE007495031884207D10549091F0968D1
:100AE00041F47021024A121F116070470800024051
:100AF000080402401AB103680B43036002E0036874
:100B00008B430360704710B50022026847F6F0730C
:100B10009A430C6A8B6823430C6923434C69234333
:100B20008C692343CC6923434C6A23438C6A234357
:100B30001A430260CB6843600B6883604B68C360F4
:100B400010BD704710B5024607E0002101E04B1CC4
:100B500099B241F270739942F9DB1300A2F10104DA
:100B6000A2B2F2D110BD4FF0E0231A6900210CE0CF
:100B700008E04FF0E0231B69934203D04FF0E023DD
:100B80001A6900E0F5E700BF491C8142F0DB7047BD
:100B900001461CE000BF00BF00BF00BF00BF00BF98
:100BA00000BF00BF00BF00BF00BF00BF00BF00BF4D
:100BB00000BF00BF00BF00BF00BF00BF00BF00BF3D
:100BC00000BF00BF00BF00BF00BF00BF00BF0A00E2
:100BD000A1F1010399B2DDD17047000030B50446A0
:100BE00004254FF4302000F06FF80546042D17D18E
:100BF0000C48006940F002000A4908610846446157
:100C0000006940F0400008614FF4302000F05CF8CB
:100C100005460448006941F6FD7108400149086134
:100C2000284630BD0020024004200B49C96811F05D
:100C3000010F01D001200EE00749C96811F0040F2F
:100C400001D0022007E00449C96811F0100F01D05B
:100C5000032000E0042070470020024003480069A0
:100C600040F0800001490861704700000020024008
:100C700070B504460D460426F00200F025F806463D
:100C8000042E11D10948006940F0010007490861AC
:100C90002580F00200F018F806460448006941F685
:100CA000FE71084001490861304670BD00200240D5
:100CB000024803494860034848607047230167457C
:100CC00000200240AB89EFCD00B502460423FFF7B8
:100CD000ABFF034603E0FFF7A7FF0346521E012BBD
:100CE00001D1002AF7D102B90523184600BD000042
:100CF0002DE9F043ADF26C4D064606EB460000EBE5
:100D0000C6012B4800EB8100D0F8248006EB46009A
:100D100000EBC601264800EB8100D0F828904F4632
:100D200045460DF2044000F001FD20E0B5F5806F6E
:100D300011D94FF48062394601A802F0E3FD4FF467
:100D4000806201A90DF2044000F002FD07F5806702
:100D5000A5F580650BE0AAB2394601A802F0D2FDE4
:100D60002A4601A90DF2044000F0F2FC0025002DF6
:100D7000DCD10DF2044000F071FC002413E006EB1E
:100D8000460000EBC6010A4800EB81001430015D0B
:100D90000DF25C40005D814204D000200DF26C4DEC
:100DA000BDE8F083641C102CE9DB0120F6E70000AD
:100DB0001A22002010B500F017F809480068094908
:100DC00088420BD04FF478610548FFF7EAF90548EF
:100DD0000349086000F014F8012010BD0020FCE772
:100DE00012220020F8DEBC8A10B5044C4FF4786261
:100DF0000021204602F086FD10BD000012220020D6
:100E000010B5044C4FF478620021204602F0EEFD4C
:100E100010BD00001222002070B50646002446E0F6
:100E200004EB440000EBC401254800EB8100416A5B
:100E300004EB440000EBC40206F1080000EB820062
:100E4000406A814200D037E0002516E004EB440000
:100E500000EBC4011A4800EB81001430415D04EB43
:100E6000440000EBC40206F1080000EB82001430DD
:100E7000405D814200D002E06D1C102DE6DB00BF1A
:100E8000102D00D018E004EB440202EBC40306F17D
:100E9000080202EB830104EB440202EBC403084A9C
:100EA00002EB8300FFF794F900B105E0641C0448ED
:100EB00008384068A042B3D800BF204670BD00008B
:100EC0001A2200202DE9F0410246002500260020CC
:100ED00000230024002791F803C00CF00F0591F8BF
:100EE00003C01CF0100F03D091F802C04CEA0505B6
:100EF00091F800C0BCF1000F31D0146800202BE045
:100F00004FF0010C0CFA00F3B1F800C00CEA030634
:100F10009E4220D183004FF00F0C0CFA03F7BC4324
:100F200005FA03FC4CEA040491F803C0BCF1280F55
:100F300006D14FF0010C0CFA00FCC2F814C00AE014
:100F400091F803C0BCF1480F05D14FF0010C0CFA29
:100F500000FCC2F810C0401C0828D1D31460B1F8BE
:100F600000C0BCF1FF0F34DD546800202EE000F11A
:100F7000080C4FF0010808FA0CF3B1F800C00CEAB5
:100F800003069E4221D183004FF00F0C0CFA03F7A9
:100F9000BC4305FA03FC4CEA040491F803C0BCF11D
:100FA000280F05D100F1080C08FA0CF8C2F81480DB
:100FB00091F803C0BCF1480F07D100F1080C4FF0C5
:100FC000010808FA0CF8C2F81080401C0828CED39B
:100FD0005460BDE8F08141617047016170472DE9BF
:100FE000F04105468846174600246EE057B105F1EA
:100FF000080108194146FFF7EBF8002863D12046A5
:10100000BDE8F08100265BE004EB440000EBC40186
:1010100005F1080000EB8100805D2E284ED1C6F15D
:101020001400032849DB04EB440000EBC40105F184
:10103000080000EB8101701C085C42280BD004EB17
:10104000440000EBC40105F1080000EB8101701CB5
:10105000085C622832D104EB440000EBC40105F1C6
:10106000080000EB8101B01C085C49280BD004EBA0
:10107000440000EBC40105F1080000EB8101B01C45
:10108000085C69281AD104EB440000EBC40105F1A7
:10109000080000EB8101F01C085C4E280BD004EB2B
:1010A000440000EBC40105F1080000EB8101F01CD5
:1010B000085C6E2802D12046A2E703E0701CC6B28D
:1010C000142EA1DB00BF601CC4B26868A0428DD89A
:1010D0004FF0FF3094E73EB55824684600F010F812
:1010E000002503E01DF8050044406D1C0C2DF9DBC4
:1010F00004B95824FF2C00D1852420463EBD0000B1
:101100000021064A00BF05E013780370401C521C02
:101110004B1CD9B20C29F7DB70470000E8F7FF1F22
:10112000024602B97047002008E0131804D0054BAE
:1011300053F821301B5C1354431CD8B20C28F4DB49
:1011400000BFEFE76C0000201748008817490880AF
:1011500008460088802804DC4FF4006014490880A9
:1011600003E04FF4006012490880114800881149DB
:10117000084411490860084600680D490988084478
:101180000E490860084600680949098808440C4966
:101190000860084600884005400D04D008460068F5
:1011A00000F5806008607047E0F7FF1FA600002090
:1011B000A4000020003C0008980000209C000020B3
:1011C000A00000200948C0880849898808430749C9
:1011D00049880843054909880843054908800846A5
:1011E000018804A001F01CFE00BFFEE70000002003
:1011F0000C0000200D0A5B4846483D253034785DE0
:101200000D0A00002DE9F043ADF6740D074688463F
:101210004FF000090DF60C0000F088FA00250024BC
:1012200018E02B490968081900F0E6FC0646284634
:101230006D1C03A90E54320A28466D1C0A54B5F5DC
:10124000006F06D14FF400620DF60C0000F080FA3A
:101250000025A41CBC42E4D32DB12A4603A90DF6F7
:101260000C0000F075FA0DF60C0000F0F7F91848C4
:101270003A4618A1036803A801F0E2FD00240BE040
:101280000DF66400025D19A101A801F0D9FD01A9C4
:1012900003A8FEF791FF641C102CF1DB15A103A835
:1012A000FEF78AFF03A800F09DF900240CE018F86F
:1012B00004100DF66400005D814204D000200DF69C
:1012C000740DBDE8F083641C102CF0DB0120F6E700
:1012D000A000002046696C6553697A653D25642C41
:1012E000253038782C20204D44353D0025303258AB
:1012F000000000000D0A000070B504460D460748C6
:1013000084420AD1064802882946064800F076FA47
:1013100006463146034801F0B9FC70BD50435441C4
:10132000A4000020AE21002070B504460548844288
:1013300007D1054800F094FA05462946024801F015
:10134000A5FC70BD50435441AE2100202DE9F04F63
:10135000A1B08046444620687D49884208D0206874
:101360007C49884204D04FF0FF3021B0BDE8F08FB7
:101370002079802802D06FF00100F6E776A11DA841
:1013800001F05EFDA11D1DA8FEF722FF10B16FF058
:101390000200EAE794F805A0208B0190BAF1000F53
:1013A00025D10198142802D06FF00300DDE7C34671
:1013B00010220BF11A016948FEF7DAFED846DBF875
:1013C0002A00674908600846006810B96FF00400F9
:1013D000CBE70020634908606349086063490860FF
:1013E000206860490968FFF787FF0120BDE7BAF16F
:1013F000020F7DD14746002608E05848815D07F17D
:101400001A00805D814200D002E0761C102EF4DBD1
:1014100000BF102E08DA56A000F0E4F82068FFF7AD
:1014200083FF6FF00500A0E7D7F82E50D7F82A0009
:101430000290022D0CD34B4902980968884207D1CB
:1014400048480068291846480068801C814208D92D
:101450004CA000F0C7F82068FFF766FF6FF00600A9
:1014600083E7AD1E2A4607F13201002002F03AF868
:10147000814607F13200691C405C00021C9007F1B4
:101480003200405D1C99084480B21C901C9949456B
:101490000AD044A000F0A6F8206832490968FFF796
:1014A0002BFF6FF0070060E72E48006810B900209E
:1014B00002F056FB2068274988420DD1002609E03A
:1014C00007F13200805D3D490978484007F132015B
:1014D0008855761CAE42F3D307F1320229462148E3
:1014E000006800F0A3F82148006828441F4900E084
:1014F0002CE008601B48006828441A4908601B4813
:10150000006817490968884210DB144914480068CC
:10151000FFF778FE40B92AA000F064F82068FFF7D2
:1015200003FF6FF0080020E700201EE70D482AA106
:10153000026803A801F084FC03A800F053F82068B7
:1015400008490968FFF7D8FE02200EE700BF0CE744
:10155000464F54415043544130000000E000002009
:1015600030000020380000203C0000203400002023
:101570004D4435204D6F64696679215265444F2191
:101580000D0A00004C656E677468206F72204F660C
:1015900066736574206572726F72215265444F21C3
:1015A0000D0A0000436865636B2043524320657257
:1015B000726F72215265444F210D0A0029000020EC
:1015C000436865636B204D4435206572726F7221EC
:1015D0005265444F210D0A004842443D25640D0ADE
:1015E0000000000070B505462C460A20FFF7BBFA44
:1015F0000BA001F015FC0BE021780B4801F0ADF9D0
:1016000000BF4021084801F0DAF80028F9D0641C36
:1016100020780028F0D10A20FFF7A5FA70BD00005D
:101620005B4941505D000000003801402DE9F04168
:1016300004460D461646002714F0010F02D0002084
:10164000BDE8F081AAB2044909680819314601F0E1
:10165000B1FB0120F4E70000A00000202DE9F041DB
:1016600090B0044620680E9060680F902088C0F308
:10167000C507382F02DAC7F1380001E0C7F178005A
:10168000804642462849204600F062F800260025A0
:1016900018E004F11800E91C405C020604F118008F
:1016A000A91C405C42EA004204F11800691C405C3D
:1016B00042EA002004F11801495D08434DF8260074
:1016C000761C2D1D0E2EE4D3694604F1080000F0AF
:1016D000CBFB0026002521E004F1080010F82610BD
:1016E00050304155503830F82600C0F3072204F13D
:1016F0005800691C4254503850F82600C0F3074285
:1017000004F15800A91C4254503850F82600000E2D
:1017100004F15801EA1C8854761C2D1D042EDBD3DD
:1017200010B0BDE8F0810000B33B0008002141602B
:10173000016005498160054AC260CA430261034AEB
:10174000D2434261704700000123456789ABCDEF6A
:101750002DE9F04391B004460F4615462088C0F3AA
:10176000C509206800EBC5002168884202D2606884
:10177000401C6060206800EBC5002060606800EBE2
:101780005570606033E017F8012B484609F10109F4
:1017900004F118010A54B9F1400F28D14FF00008A4
:1017A00000261AE004F11800F11C405C020604F166
:1017B0001800B11C405C42EA004204F11800711CA0
:1017C000405C42EA002004F11801895D084301A948
:1017D00041F8280008F10108361DB8F1100FE1D3D7
:1017E00001A904F1080000F03FFB4FF000092800B8
:1017F000A5F10105C7D111B0BDE8F0832DE9F04195
:1018000004460E461746254632212846FEF7C9FCF7
:101810000F48286080202871022068710DA1A81D42
:1018200001F00EFB0C480088401C80B20A49088079
:10183000E882182028831022084905F11A00FEF7D3
:1018400097FCC5F82A60C5F82E703220BDE8F081FB
:1018500050435441300000002C000020E0000020E4
:1018600070B5044625462C212846FEF79AFC0D4803
:10187000286080202871002068710BA1A81D01F04C
:10188000DFFA0A480078E8821220288308A105F1CF
:101890001A00FEF7ABFC00206885074908802C2061
:1018A00070BD00005043544130000000290000206A
:1018B0004E554C4C000000002C0000202DE9F0415A
:1018C00004460E4617469846254650212846FEF700
:1018D00068FC0F482860952028710420687100205A
:1018E000E88236202883A5F8466006EB460000EB28
:1018F000C602084800EB82012C2205F11A00FEF70F
:1019000037FCC5F84C80AF645020BDE8F081000082
:10191000504354411A22002070B504462546222126
:101920002846FEF73EFC09482860952028710320D0
:1019300068710020E882082028835A20A883142098
:1019400068830348C5F81E00222070BD50435441EF
:1019500000F01F0000BFFEE77047000070B50021D7
:1019600000230F22C4780CB3164C246804F4E064FE
:10197000C4F5E064210AC1F10403CA40447804FAC2
:1019800003F184781440214309010F4C0678A155D6
:10199000047804F01F050124AC4005786D114FF068
:1019A000E02606EB8505C5F8004109E0047804F05F
:1019B0001F050124AC40054D0678761145F82640F8
:1019C00070BD00000CED00E000E400E080E100E00C
:1019D00002490143024A1160704700000000FA0505
:1019E0000CED00E004490978044A117002490870BE
:1019F0000121034A51717047270000202800002070
:101A00002000002029B1064A52690243044B5A6162
:101A100004E0034A52698243014B5A617047000057
:101A20000010024029B1064A92690243044B9A61B0
:101A300004E0034A92698243014B9A6170470000B7
:101A40000010024030B500210022002400232D4D5B
:101A50006D6805F00C0121B1042905D0082923D1B6
:101A600005E0294D056022E0284D05601FE0254D69
:101A70006D6805F47012234D6D6805F480340225FD
:101A800005EB92421CB9224D554305600BE01D4DFC
:101A90006D6815F4003F03D01E4D5543056002E00C
:101AA0001A4D5543056002E0174D056000BF00BFA9
:101AB000144D6D6805F0F0010909174D6B5C056860
:101AC000DD4045600F4D6D6805F4E061090A124D77
:101AD0006B5C4568DD4085600A4D6D6805F46051BA
:101AE000C90A0D4D6B5C4568DD40C560054D6D68EC
:101AF00005F44041890B094D6B5CC568B5FBF3F5F6
:101B0000056130BD0010024000127A00001BB700D2
:101B100000093D00808D5B00A8000020B800002077
:101B2000F0B505460B461646002700240DE028199F
:101B300000F062F8024638467F1C1A544FEA122C15
:101B400038467F1C03F800C0A41CB442EFDBF0BD94
:101B500021B1028842F04002028004E002884FF680
:101B6000BF731A40028070470246002013890B425F
:101B700001D0012000E000207047014688897047AD
:101B80008181704710B50022028802F441520B880F
:101B90004C8823438C882343CC8823430C892343DC
:101BA0004C8923438C892343CC8923431A430280E5
:101BB000838B4FF2FF74234083830B8A038210BD13
:101BC00010B5044600BF02210A48FFF7CDFF0028E8
:101BD000F9D021460748FFF7D3FF00BF0121054890
:101BE000FFF7C2FF0028F9D00248FFF7C6FFC0B2D6
:101BF00010BD000000300140014608887047704762
:101C000010B500F001F810BD0CB500200190009057
:101C10003048006840F480302E49086000BF2D48ED
:101C2000006800F4003000900198401C019000987A
:101C300018B90198B0F5A06FF1D12648006810F4EA
:101C4000003F02D00120009001E0002000900098A9
:101C500001283ED12048006840F010001E4908606D
:101C60000846006820F00300086008460068086025
:101C70001848406817494860084640684860084668
:101C8000406848600846406820F47C104860084678
:101C9000406840F4302048600846006840F080709A
:101CA000086000BF0B48006810F0007FFAD00948B8
:101CB000406820F00300074948600846406840F04B
:101CC0000200486000BF0348406800F00C0008288C
:101CD000F9D10CBD001002400020024030B5024690
:101CE0000B461946144607E008782578A84201D02B
:101CF000012030BD491C641C08780028F4D100BFC5
:101D0000F7E7000010B5002012490860124908608A
:101D100012480078122806D0342805D0562807D05B
:101D2000782814D107E012E00D48FFF7FDFA0EE025
:101D3000FEF714FC0BE0FEF77BFB0A48FFF752FCB2
:101D400001F09AFB01F0D4FA01F0E8FC00BF00BFFB
:101D500010BD00001400002010000020270000200B
:101D600050435441A43B000801200749C87007486C
:101D70000068401C05490860322804DB0020086028
:101D80000120014908717047200000200800002050
:101D900010B51348006840F001001149086008467A
:101DA0004068104908400E494860084600680E49DE
:101DB00008400B4908600846006820F4802008604D
:101DC0000846406820F4FE0048604FF41F00886019
:101DD000FFF716FF4FF000600449086010BD0000D7
:101DE000001002400000FFF8FFFFF6FE08ED00E0E3
:101DF00010B517480068401C04D015480068401C06
:101E00001349086013480078122806D034280CD0F3
:101E100056280BD0782818D109E00D480068012811
:101E200002D17820FFF7DEFD0FE00EE00DE008485C
:101E30000068042800D210BD0548007810F0010F9A
:101E400002D005A0FFF7CEFB00BF00BF00BFF2E746
:101E500014000020270000204E6F20417070210DDB
:101E60000A00000070470000F0B505460C462868DF
:101E70006968AA68EB6801EA020623EA01073E43A3
:101E800027683E44FE4F3E443044C60146EA506057
:101E9000084400EA010622EA00073E4367683E4420
:101EA000F84F3E4433441E0346EA1353034403EA07
:101EB000000621EA03073E43A7683E44F24F3E4432
:101EC0003244560446EAD2321A4402EA030620EAB1
:101ED00002073E43E7683E44EC4F3E4431448E05E2
:101EE00046EA9121114401EA020623EA01073E4332
:101EF00027693E44E64F3E443044C60146EA5060FE
:101F0000084400EA010622EA00073E4367693E44AE
:101F1000E04F3E4433441E0346EA1353034403EAAE
:101F2000000621EA03073E43A7693E44DA4F3E44D8
:101F30003244560446EAD2321A4402EA030620EA40
:101F400002073E43E7693E44D44F3E4431448E0588
:101F500046EA9121114401EA020623EA01073E43C1
:101F6000276A3E44CE4F3E443044C60146EA5060A4
:101F7000084400EA010622EA00073E43676A3E443D
:101F8000C84F3E4433441E0346EA1353034403EA56
:101F9000000621EA03073E43A76A3E44A6F524460D
:101FA0004F3E3244560446EAD2321A4402EA03064D
:101FB00020EA02073E43E76A3E44BB4F3E443144B9
:101FC0008E0546EA9121114401EA020623EA01073F
:101FD0003E43276B3E44B54F3E443044C60146EA7B
:101FE0005060084400EA010622EA00073E43676B9E
:101FF0003E44AF4F3E4433441E0346EA135303446A
:1020000003EA000621EA03073E43A76B3E44A94FBB
:102010003E443244560446EAD2321A4402EA0306E7
:1020200020EA02073E43E76B3E44A34F3E4431445F
:102030008E0546EA9121114401EA030622EA0307CC
:102040003E4367683E449D4F3E443044460146EA65
:10205000D060084400EA020621EA02073E43A7696D
:102060003E44974F3E4433445E0246EAD353034412
:1020700003EA010620EA01073E43E76A3E44914F26
:102080003E443244960346EA92421A4402EA00066B
:1020900023EA00073E4327683E448B4F3E443144C9
:1020A0000E0546EA1131114401EA030622EA03074C
:1020B0003E4367693E44854F3E443044460146EA0C
:1020C000D060084400EA020621EA02073E43A76AFC
:1020D0003E447F4F3E4433445E0246EAD3530344BA
:1020E00003EA010620EA01073E43E76B3E44794FCD
:1020F0003E443244960346EA92421A4402EA0006FB
:1021000023EA00073E4327693E44734F3E4431446F
:102110000E0546EA1131114401EA030622EA0307DB
:102120003E43676A3E446D4F3E443044460146EAB2
:10213000D060084400EA020621EA02073E43A76B8A
:102140003E44674F3E4433445E0246EAD353034461
:1021500003EA010620EA01073E43E7683E44614F77
:102160003E443244960346EA92421A4402EA00068A
:1021700023EA00073E43276A3E445B4F3E44314416
:102180000E0546EA1131114401EA030622EA03076B
:102190003E43676B3E44554F3E443044460146EA59
:1021A000D060084400EA020621EA02073E43A7681D
:1021B0003E444F4F3E4433445E0246EAD353034409
:1021C00003EA010620EA01073E43E7693E44494F1E
:1021D0003E443244960346EA92421A4402EA00061A
:1021E00023EA00073E43276B3E44434F3E443144BD
:1021F0000E0546EA1131114481EA02065E40676924
:102200003E443E4F3E443044060146EA10700844C6
:1022100080EA01065640276A3E44394F3E44334423
:10222000DE0246EA5353034483EA00064E40E76A5F
:102230003E44344F3E443244160446EA12421A44A5
:1022400082EA03064640A76B3E442F4F3E4431448A
:10225000CE0546EA5121114481EA02065E406768D4
:102260003E442A4F3E443044060146EA107008447A
:1022700080EA0106564027693E44254F3E4449E026
:1022800078A46AD756B7C7E8DB702024EECEBDC16C
:10229000AF0F7CF52AC68747134630A8019546FD47
:1022A000D8988069AFF7448BBED75C892211906BB8
:1022B000937198FD8E4379A62108B44962251EF6D4
:1022C00040B340C0515A5E26AAC7B6E95D102FD66A
:1022D0005314440281E6A1D8C8FBD3E7E6CDE1213F
:1022E000D60737C3870DD5F4ED145A4505E9E3A9A0
:1022F000F8A3EFFCD9026F678A4C2A8D4239FAFFA6
:1023000081F6718722619D6D0C38E5FD44EABEA41B
:10231000A9CFDE4B3344DE0246EA5353034483EA3B
:1023200000064E40E7693E449F4F3E443244160447
:1023300046EA12421A4482EA03064640A76A3E442D
:102340009A4F3E443144CE0546EA5121114481EA78
:1023500002065E40676B3E44954F3E4430440601A2
:1023600046EA1070084480EA0106564027683E4459
:10237000904F3E443344DE0246EA5353034483EA1B
:1023800000064E40E7683E448B4F3E4432441604FC
:1023900046EA12421A4482EA03064640A7693E44CE
:1023A000864F3E443144CE0546EA5121114481EA2C
:1023B00002065E40676A3E44814F3E443044060157
:1023C00046EA1070084480EA01065640276B3E44F6
:1023D0007C4F3E443344DE0246EA5353034483EACF
:1023E00000064E40E76B3E44774F3E4432441604AD
:1023F00046EA12421A4482EA03064640A7683E446F
:10240000724F3E443144CE0546EA5121114461EAFF
:102410000306564027683E446D4F3E4430448601D3
:1024200046EA9060084460EA02064E40E7693E448E
:10243000684F3E4433449E0246EA9353034463EAA2
:1024400001064640A76B3E44634F3E443244D603E8
:1024500046EA52421A4462EA00065E4067693E4418
:102460005E4F3E4431444E0546EAD121114461EAB3
:1024700003065640276B3E44594F3E443044860184
:1024800046EA9060084460EA02064E40E7683E442F
:10249000544F3E4433449E0246EA9353034463EA56
:1024A00001064640A76A3E444F4F3E443244D6039D
:1024B00046EA52421A4462EA00065E4067683E44B9
:1024C0004A4F3E4431444E0546EAD121114461EA67
:1024D00003065640276A3E44454F3E443044860139
:1024E00046EA9060084460EA02064E40E76B3E44CC
:1024F000404F3E4433449E0246EA9353034463EA0A
:1025000001064640A7693E443B4F3E443244D60351
:1025100046EA52421A4462EA00065E40676B3E4455
:10252000364F3E4431444E0546EAD121114461EA1A
:102530000306564027693E44314F3E4430448601ED
:1025400046EA9060084460EA02064E40E76A3E446C
:102550002C4F3E4433449E0246EA9353034463EABD
:1025600001064640A7683E44274F3E443244D60306
:1025700046EA52421A4462EA00065E40676A3E44F6
:10258000224F3E4431444E0546EAD12111442E6883
:1025900006442E606E680E446E60AE681644AE60EF
:1025A000EE681E44EE60F0BD604BBBF670BCBFBE73
:1025B000C67E9B28FA27A1EA8530EFD4051D880442
:1025C00039D0D4D9E599DBE6F87CA21F6556ACC4B6
:1025D000442229F497FF2A43A72394AB39A093FC04
:1025E000C3595B6592CC0C8F7DF4EFFFD15D848580
:1025F0004F7EA86FE0E62CFE144301A3A111084E04
:10260000827E53F735F23ABDBBD2D72A91D386EBFF
:102610001CB540F22441434800F0DEF840B3414885
:10262000008801903F48001D008801903E48C06D21
:1026300041F25201081A019000213B485830FEF740
:10264000A7F93A48007850B939493A48019AFDF754
:102650008FFD39490198088001203449087041F202
:1026600052003149C86501212F485830FEF790F9D2
:1026700040F225512B4800F0AFF8002842D02948FD
:1026800000F066F9C0B2009040F22551254800F0F4
:1026900072F82A48008818B10020294908801CBD1A
:1026A0009DF80010264802880088401C244B1880A2
:1026B0001F4881540078892814D1184600880328BF
:1026C00015DB1B488078C01C0190184600880199D2
:1026D00088420CD318460088184908800020194603
:1026E000088004E000201649088011490870144849
:1026F000008841F25101884204DB00201049088023
:102700000E49088008210F4800F059F8012806D129
:10271000044800F01DF90821024800F023F800BF2A
:10272000BDE700000038014000000240200000200A
:102730005C1100200A010020400000204E00002013
:102740004C000020004800407047704710B5FFF76C
:102750005FFF10BD10B5FFF7F7FF10BD10B5FFF715
:10276000F4FF10BD01F40072B2F5007F00D100BF8C
:10277000CA430280704710B500220023A1F51064FF
:102780006A3C00D100BF0A1201249440A3B2DC438A
:10279000048010BD21B1828942F40052828104E09C
:1027A00082894DF6FF731A40828170471AB1838A7D
:1027B0000B43838202E0838A8B4383827047024605
:1027C0000020B1F5007F00D100BF13880B4201D07B
:1027D000012000E00020704770B50246002400236D
:1027E00000250020A1F510666A3E00D100BFC1F3AC
:1027F000421501F01F03012606FA03F3012D02D151
:102800009689334006E0022D02D1168A334001E05A
:10281000968A33400C12012606FA04F416883440D6
:1028200013B10CB1012000E0002070BDF0B50346EB
:102830000024002600250020A1F510676A3F00D182
:1028400000BF1846C1F3421401F01F06012707FA22
:1028500006F5012C01D10C3004E0022C01D110301E
:1028600000E014301AB107682F43076002E00768E0
:10287000AF430760F0BD00002DE9F04786B0054684
:102880000E460024A24600BFA1460027B08900B131
:1028900000BF2F462C8A4CF6FF700440F08804439A
:1028A0002C82AC894EF6F3100440B088318908437D
:1028B000718908430443AC81AC8A4FF6FF40044061
:1028C000B0890443AC8201A8FFF7BCF81F488742D7
:1028D00002D1DDF810A001E0DDF80CA0A88910F409
:1028E000004F08D00AEBCA0000EB0A10316849001B
:1028F000B0FBF1F807E00AEBCA0000EB0A10316800
:102900008900B0FBF1F86420B8FBF0F00401200965
:10291000642101FB1089A88910F4004F08D03220EF
:1029200000EBC900B0FBF1F000F00700044308E041
:10293000322000EB09106421B0FBF1F000F00F0031
:1029400004432C8106B0BDE8F08700000038014048
:1029500001468888C0F308007047C1F308028280EE
:102960007047000000B58DB001210846FFF74AF816
:102970002B48FEF719F82B4801902B4802901020A5
:102980000390642004900020059080200690002091
:102990000790089009900A900B9001A92048FEF733
:1029A000B2F80E208DF8300003208DF8310002209F
:1029B0008DF8320001208DF833000CA8FEF7CEFF11
:1029C000012202211648FEF795F800211448FDF770
:1029D000DFFF13481430FDF7E7FF1248019013485A
:1029E00002900020039041F25200049000200590D4
:1029F0008020069000200790089009904FF4005026
:102A00000A9000200B9001A905481430FEF77BF8CE
:102A1000012103481430FDF7BBFF0DB000BD0000DD
:102A20004400024004380140AE2100205C11002027
:102A300000B587B0012144F20400FEF7F3FF4FF424
:102A40000070ADF8140018208DF8170003208DF8E1
:102A5000160005A92E48FEF735FA4FF48060ADF850
:102A6000140004208DF8170003208DF8160005A926
:102A70002748FEF727FA4FF4E13001900020ADF827
:102A80000800ADF80A00ADF80C00ADF810000C20FD
:102A9000ADF80E0001A91F48FFF7EEFE01211D4809
:102AA000FFF778FE4FF4E060FEF792FF25208DF8E7
:102AB000180000208DF819008DF81A0001208DF8FB
:102AC0001B0006A8FEF74AFF40211248FFF74AFE06
:102AD000002240F227710F48FFF7A8FE002240F2C3
:102AE00025510C48FFF7A2FE012240F2244109487B
:102AF000FFF79CFE012240210648FFF757FE002207
:102B000080210448FFF752FEFFF72CFF07B000BDFD
:102B1000000801400038014010B53F4800781228F5
:102B20001BD13EA14148FFF7D9F830B93420FEF758
:102B300059FF3FA0FEF756FD0EE041A13B48FFF7CD
:102B4000CDF830B95620FEF74DFF41A0FEF74AFD03
:102B500002E044A0FEF746FD10BD2F48007834285F
:102B600004D02D480078562800D0F5E72F4800788B
:102B700050280BD12D484078432807D12B48807826
:102B8000542803D12948C078412800D0E4E72748D9
:102B9000007980281DD1354801882448FEF7D6FBEE
:102BA00004464CB9012000F0DBFF31A0FEF71AFD0E
:102BB0005620FEF717FFCFE714F1020F2ADA14F1BF
:102BC000060F27DD2DA0FEF70DFD7820FEF70AFF8A
:102BD00020E01648007995281CD124480188134824
:102BE000FDF7C8FC04464CB921A0FEF7FBFC782099
:102BF000FEF7F8FE012024490870ADE714F1020F3A
:102C000008DA14F1060F05DD1CA0FEF7EBFC7820B6
:102C1000FEF7E8FE00BF9FE727000020444F574E15
:102C20004C4F41445F415050000000000A01002019
:102C3000444F574E4C4F41445F4150500D0A0000E5
:102C4000444F574E4C4F41445F5246494C45530008
:102C5000444F574E4C4F41445F5246494C45530DEB
:102C60000A0000002D2D2D2D0D0A0000400000202F
:102C7000436F6D706C65746564210000494150209C
:102C800053746F70210D0A006400002070B5054672
:102C90000E4600240BE0295D0648FFF75EFE00BFEC
:102CA00040210448FFF78BFD0028F9D0641CB44292
:102CB000F1DB70BD0038014000BFFEE710B586B003
:102CC00000F036F810211848FEF787F90020ADF81B
:102CD00004004FF48270ADF806000020ADF8080043
:102CE0000220ADF80A000120ADF80C004002ADF85A
:102CF0000E000820ADF810000020ADF812000720EB
:102D0000ADF8140001A90948FEF73CFF012107486E
:102D1000FEF71EFF4FF47A70FDF73AFF00F020FE39
:102D20000446012006B010BD0008014000300140FB
:102D300008B501210420FEF775FE01210803FEF706
:102D400071FE2020ADF8000003208DF8020018204D
:102D50008DF8030069461548FEF7B4F88020ADF8F9
:102D6000000069461148FEF7ADF84020ADF80000BC
:102D700004208DF8030069460C48FEF7A3F81020E4
:102D8000ADF800008DF8030069460848FEF79AF890
:102D90001020ADF800008DF8030069460448FEF7E6
:102DA00091F810210248FEF718F908BD000801400B
:102DB000001001402DE9F04705460E469046B5F15A
:102DC000006F07D3154800884FF0006101EB8020A9
:102DD000A84201D8BDE8F087A805800D00D0F9E72A
:102DE000FDF766FF2846FDF7F9FE0746042F00D0E1
:102DF000F0E700240CE0315D601C305C01EB00204A
:102E00001FFA80F928194946FDF732FFA01C84B249
:102E10004445F0DBFDF722FF00BFDBE7A600002002
:102E20000FB4054B10B503A9044A029800F02CF822
:102E300010BC5DF814FB0000F9360008DC0000202F
:102E40000FB4084B10B504A902AA039800F01CF8AF
:102E5000044602A9002000F046FA204610BC5DF8A6
:102E600014FB0000E732000802E008C8121F08C186
:102E7000002AFAD170477047002001E001C1121FFB
:102E8000002AFBD1704700002DE9FF4F8DB00F469F
:102E900005460026DEE1252874D100246D1CF14989
:102EA000A246A14601222B78203B02FA03F00842F9
:102EB00002D004436D1CF6E728782A2810D06FF062
:102EC0002F022878A0F13001092915D80AEB8A01D0
:102ED00002EB410144F0020400EB010A6D1CF0E733
:102EE00057F804ABBAF1000F03DA44F40054CAF106
:102EF000000A44F002046D1C28782E2817D115F81A
:102F0000010F44F004042A280ED06FF02F02287815
:102F1000A0F1300109290AD809EB890102EB41012E
:102F200000EB01096D1CF2E757F8049B6D1C287833
:102F30006C280FD006DC4C2817D068280DD06A28E2
:102F400014D104E0742810D07A280FD10DE044F495
:102F500000140AE044F4801401E044F44014697859
:102F6000814202D16D1C04F580146D1C2A786E2AF2
:102F700020D00DDC632A33D005DC002A6FD0582A1C
:102F800012D1A2E011E0642A6AD0692A0CD167E06C
:102F9000732A2FD004DC6F2A6FD0702A04D199E0F5
:102FA000752A6BD0782A6AD01046DDE90F12904757
:102FB000761C4EE1C4F30250022806D003280AD042
:102FC000042801CF0AD0066043E101CF4FEAE67141
:102FD000C0E900613DE101CF06803AE1067038E1C9
:102FE00017F8040B8DF8000000208DF80100EB4667
:102FF000012003E057F804BB4FF0FF3061074FF0AA
:10300000000102D40DE008F10101884649450FDABC
:103010008045F8DB1BF808100029F4D108E008F11E
:10302000010188468142FADB1BF808100029F6D11D
:10303000DDE90F23AAEB08008146214600F03BF9A9
:10304000304400EB080604E0DDE90F121BF8010B29
:103050009047B8F10108F7D221464846F4E0FDE078
:103060000A21C4F302534FF0000B0891022B07D042
:1030700001CFC117032B09D00AE034E023E024E09C
:10308000FF1D27F00707F7E8020105E000B2C117AE
:10309000042B01D140B2C117002907DA4FF0000C10
:1030A000D0EB0C006CEB01012D2302E0230504D5CD
:1030B0002B238DF82430012303E0E30701D02023E4
:1030C000F7E7984650E00A210EE010204FF0000B81
:1030D00008900CE010214FF0000B44F004044FF076
:1030E0000809089103E008214FF0000B0891C4F390
:1030F0000253022B04D001CF0021032B06D006E09F
:10310000FF1D27F00707F7E8020103E080B2042B58
:1031100000D1C0B24FF00008230725D5702A2AD06D
:10312000DDF820C08CF0100C5CEA0B0C09D150EAE1
:10313000010306D030238DF824308DF8252002239A
:103140009846DDF820C08CF0080C5CEA0B0C0BD123
:1031500050EA010301D1630706D530238DF82430EE
:103160004FF00108A9F10109582A09D03EA20B929B
:1031700008AA0A9211E040238DF824300123DFE7EA
:103180003EA2F4E75B46089AFDF739F80B9B9B5C7F
:103190000A9AA2F101020A92137050EA0102F1D1D7
:1031A0000A98ADEB000000F1200B600702D524F473
:1031B000803401E04FF00109D94502DDA9EB0B0095
:1031C00000E0002000EB0B0141440890AAEB010A4B
:1031D000E00306D4DDE90F232146504600F06BF8EA
:1031E0000644002008E009A911F80900DDE90F12E2
:1031F0009047761C09F1010081464045F3DBE0036E
:103200000CD5DDE90F232146504600F054F8064462
:1032100004E0DDE90F1230209047761C0899481E23
:1032200008900029F5DC08E00A980A990078491C02
:103230000A91DDE90F129047761CBBF10001ABF15A
:10324000010BF1DC21465046DDE90F2300F020F8A8
:1032500006446D1C287800287FF41DAE11B030465E
:10326000BDE8F08F0928010030313233343536376C
:1032700038396162636465660000000030313233C2
:103280003435363738394142434445460000000062
:103290002DE9F041044600251E461746880405D452
:1032A00006E039462020B04705F10105641EF8D537
:1032B0002846BDE8F0812DE9F041044600251E4670
:1032C0009046C80301D5302700E02027880405D5A3
:1032D00006E041463846B04705F10105641EF8D5C1
:1032E0002846BDE8F0810A68531C0B6010707047D7
:1032F00070B590B001216846FDF712FF0C216846B9
:1033000000F09AF90646342203A91E480068FEF729
:1033100007FCDDF82B00B04201D110B070BD00F009
:10332000B1FA002529E025B90C226946342000F0C5
:1033300031F8681C05461449884200D3002513481B
:10334000008800B919E01148017803AB32461048F3
:1033500000F0E6F804462CB90C226946352000F04E
:1033600019F80BE0042C04D10C226946372000F038
:1033700011F800200549088000BFD4E700BF00BF56
:10338000CBE7000098000020C0C62D004E000020B2
:103390005C1100202DE9F04F91B082468B46174614
:1033A0000DF10706F81C00F0FF08002589222946C8
:1033B0006D1C01A8425429466D1C00F801A0294645
:1033C0006D1C00F801802B480088021229466D1CF4
:1033D00001A842542748027829466D1C01A842548E
:1033E000002408E01BF804202846691CCDB201A97E
:1033F0000A54601CC4B2BC42F4DB08F10300C0B242
:103400008DF800009DF804008DF801009DF805007E
:103410008DF8020000240FE0032094FBF0F100FB84
:1034200011401DF80000315D48403055305D80F09E
:1034300086003055601CC4B2A8F10100A042EBDC4C
:103440004FF00009002405E001A8005D80EA0909A9
:10345000601CC4B2AC42F7DB2846691CCDB201A99E
:1034600001F80090294601A8FFF710FC11B0BDE853
:10347000F08F00009400002008B5042269460E4831
:103480000068FEF74DFB0D490098884202D0009875
:10349000401C00D108BD002000900CE0009810B93D
:1034A00007A0FFF7BDFC0098401C0D490090884222
:1034B00001D300200090F1E79C000020D0F1445C93
:1034C0004C61737420757064617465206572722C30
:1034D000206E656564207265747279210D0A0000A2
:1034E00000093D00F0B507460C461546002606E0EB
:1034F00014F8011B384600F007F80746761CAE4268
:10350000F6D33846F0BD0000024682EA0100C0B2A0
:10351000024B33F8100080EA22207047F43B000889
:103520002DE9F84F05468846924699464FF0000B24
:10353000EE1C2878892802D00120BDE8F88FA878F1
:10354000C01C404501D00220F7E7002404E0285DBC
:1035500080EA0B0B601CC4B2A8F10100A042F6DCAB
:10356000285C584501D00320E7E78DF800802878D3
:103570008DF8010068788DF8020000240FE0032028
:1035800094FBF0F100FB11401DF80000315D484054
:103590003055305D80F086003055601CC4B26878CC
:1035A000401EA042EBDC6878362801D00420C4E736
:1035B000B61C37783F0227F0FF07707807433F02B9
:1035C00027F0FF07B07807433F0227F0FF07F078A6
:1035D0000743C9F81F7000240CE016F8010BA97905
:1035E000484009F8040005EB0800B04200D82E4618
:1035F000601CC4B21F2CF0D300240DE016F8010BA0
:103600002979484009F12301085505EB0800B0422B
:1036100000D82E46601CC4B2112CEFD33422494688
:1036200004480068FFF7C6FB574501D1002084E736
:10363000042082E7980000202DE9F043D1B08046B5
:103640000F464FF480722B4911A8FCF791FD00261C
:10365000002408E018F80400464018F8040001A906
:103660000855601CC4B2BC42F4DB7E4011A810F8BF
:10367000069000240CE001A8005D80EA090684EAB7
:10368000060001A9085511A810F80690601CC4B2E4
:10369000BC42F0DB002413E004EB440001A9085C09
:1036A00004EB4401491C01AA515C80EA010604EBC9
:1036B0004400801C01A9085C70400855601CC4B21D
:1036C000042CE9DB9DF804502D0225F0FF059DF840
:1036D000050005432D0225F0FF059DF80600054372
:1036E0002D0225F0FF059DF807000543284651B03F
:1036F000BDE8F083F43D000870B504460D46E1B224
:103700000548FFF72AF900BF40210348FFF757F8A3
:103710000028F9D0204670BD0038014010B502489D
:10372000006800F003F810BDA000002010B50446AA
:10373000206814490840B0F1005F18D1002240F21F
:1037400024411148FFF772F8002240210E48FFF78C
:103750002DF800204FF0E021086160680B490860F7
:103760002068FCF7EFFC09480068804708E006E0A5
:1037700007A0FDF737FF4FF47A70FDF7E3F9F7E79D
:1037800010BD00000000FE2F003801404400002062
:103790004E6F204170700D0A00000000FFF748F9DD
:1037A000324800686422B0FBF2F1B1F1807F01D3AE
:1037B00001201DE021F07F40401E4FF0E0225061CB
:1037C00050170F22002807DA13071D0E284B00F0B0
:1037D0000F04241F1D5503E013071C0E254B1C541A
:1037E00000BF00204FF0E022906107201061002010
:1037F00008B100BFFEE7FDF7A7FCFFF75FFAFDF792
:10380000D9FAFDF768FC1C4908701C4800210160CA
:10381000818081711220FEF7E5F8FCF769FE24E053
:103820001648007848B1FFF777F90020134908706F
:1038300041F252011248FCF7B4FC1048407920B123
:1038400000200E494871FEF75DFA0C48C07820B19F
:1038500000200A49C870FEF705FB0848007920B12E
:10386000002006490871FEF7C3FAD9E7BC00002022
:1038700018ED00E000E400E0290000202000002016
:103880000A01002010B5002240F224410948FEF749
:10389000CDFF002240210748FEF788FF012240F2B9
:1038A00025510448FEF7C2FF002003490880034960
:1038B000088010BD003801404C0000204E00002060
:1038C00010B50446240300F0EBF800F087F810214F
:1038D0000B48FDF780FB2020FEF772F9C4F3074088
:1038E000FEF76EF9C4F30720FEF76AF9E0B2FEF7BF
:1038F00067F910210248FDF770FB00F06FF810BD6A
:10390000000801402DE9F04105460C4617461021FC
:103910001248FDF760FB0B20FEF752F9C4F3074095
:10392000FEF74EF9C4F30720FEF74AF9E0B2FEF7BE
:1039300047F9FF20FEF744F92870002605E0FF2034
:10394000FEF73EF9A855701C86B2BE42F7DB102187
:103950000248FDF742FBBDE8F0810000000801408D
:103960002DE9F041002400250026002710210F48F2
:10397000FDF731FB9F20FEF723F9FF20FEF720F92A
:103980000546FF20FEF71CF90646FF20FEF718F952
:10399000074610210548FDF720FB280440EA0620D1
:1039A00040EA07042046BDE8F0810000000801401D
:1039B00010B5002410210848FDF70DFB0520FEF787
:1039C000FFF8FF20FEF7FCF8044610210248FDF73F
:1039D00004FB204610BD00000008014010B500BFE8
:1039E000FFF7E6FF10F0010FFAD110BD2DE9F04707
:1039F00081460F4616464FEA1738C7F30B0ACAF539
:103A00008054A64200DC344644E04FEA08314FF4CB
:103A100080522248FFF776FF002508E00AEB0500F8
:103A20001E49085CFF2800D003E0681C85B2A5424F
:103A3000F4DB00BFA54216DA4046FFF741FF002540
:103A400007E019F8050005EB0A01144A5054681CF8
:103A500085B2A542F5DB4FEA08314FF480520F489A
:103A600000F02EF804E022463946484600F028F8D7
:103A7000A64200D10FE008F101084FF0000AA1446E
:103A80002744301B86B2B6F5805F02DD4FF48054C8
:103A900000E03446B9E700BFBDE8F087923100206E
:103AA00010B510210548FDF796FA0620FEF788F8B4
:103AB00010210248FDF791FA10BD000000080140F6
:103AC0002DE9F04107460E461446F0B2C0F5807568
:103AD000AC4200DC254612E02A463146384600F06A
:103AE00013F8AC4200D10BE02F442E44601B84B28B
:103AF000B4F5807F02DD4FF4807500E02546EBE7EA
:103B000000BFBDE8F08100002DE9F04106460C46FB
:103B10001746FFF7C5FF10211048FDF75CFA022099
:103B2000FEF74EF8C4F30740FEF74AF8C4F3072047
:103B3000FEF746F8E0B2FEF743F8002504E0705DBA
:103B4000FEF73EF8681C85B2BD42F8DB1021034841
:103B5000FDF743FAFFF742FFBDE8F081000801409E
:103B60001CB5044614B90C48019001E00B480190C3
:103B7000042269460A480068FDF7D2FFDDE900012A
:103B8000884200D11CBD042201A905480068FFF746
:103B900011F900BFF6E700004D318724D0F1445CF5
:103BA0009C0000204D32302D4941502D563230318D
:103BB0000D0A00800000000000000000000000006E
:103BC00000000000000000000000000000000000F5
:103BD00000000000000000000000000000000000E5
:103BE00000000000000000000000000000000000D5
:103BF000000000000000C1C081C1400101C3C0033A
:103C0000800241C201C6C006800741C70005C1C588
:103C100081C4400401CCC00C800D41CD000FC1CF48
:103C200081CE400E000AC1CA81CB400B01C9C00938
:103C3000800841C801D8C018801941D9001BC1DBD8
:103C400081DA401A001EC1DE81DF401F01DDC01D88
:103C5000801C41DC0014C1D481D5401501D7C017A8
:103C6000801641D601D2C012801341D30011C1D1B8
:103C700081D0401001F0C030803141F10033C1F3F8
:103C800081F240320036C1F681F7403701F5C03588
:103C9000803441F4003CC1FC81FD403D01FFC03F48
:103CA000803E41FE01FAC03A803B41FB0039C1F938
:103CB00081F840380028C1E881E9402901EBC02B98
:103CC000802A41EA01EEC02E802F41EF002DC1ED88
:103CD00081EC402C01E4C024802541E50027C1E7A8
:103CE00081E640260022C1E281E3402301E1C021B8
:103CF000802041E001A0C060806141A10063C1A3B8
:103D000081A240620066C1A681A7406701A5C06587
:103D1000806441A4006CC1AC81AD406D01AFC06F47
:103D2000806E41AE01AAC06A806B41AB0069C1A937
:103D300081A840680078C1B881B9407901BBC07BD7
:103D4000807A41BA01BEC07E807F41BF007DC1BD87
:103D500081BC407C01B4C074807541B50077C1B7A7
:103D600081B640760072C1B281B3407301B1C071B7
:103D7000807041B00050C190819140510193C05377
:103D8000805241920196C056805741970055C19587
:103D900081944054019CC05C805D419D005FC19F47
:103DA000819E405E005AC19A819B405B0199C05937
:103DB000805841980188C04880494189004BC18B97
:103DC000818A404A004EC18E818F404F018DC04D87
:103DD000804C418C0044C184818540450187C047A7
:103DE000804641860182C042804341830041C181B7
:103DF0008180404068596364C8CCAAA7A2ABA56E75
:103E00006A568A57F4BBFEFA26212D290D093E3A3F
:103E100037320A07F7F2FBF5FFF61C181314F1FD11
:103E2000F90C9F089A97929B959F121B152C28239B
:103E3000F92A2722242E67252F98FC75F8F33C38A1
:103E400033340304050F06017A7772626B83848E24
:103E5000C4CB8782353F364F3D399C989394424F6F
:103E60004641818D4D49717D7996919D99C3C41DBF
:103E7000CECA7F767C7873747E7B751E1A171F16E8
:103E8000111D47195DC7C2CBC5CFD1DDD94C48C67E
:103E9000C1CD61C9D78CFD88A1ADA9B1BDB98B8554
:103EA0008F4B4586DCD8D3D4DED2DBD5DFD6434476
:103EB0004E4AE747ACA8A3A4AEBA0DB7B2AFA6E48A
:103EC000EEEAE7E2E1ED0FE966616D69BBB5BFB609
:103ED000ECE80BE3525C656F5853540C5E5B555F26
:103EE000312F9A0B0B5A2B9E0289593B0E516CEBCA
:103EF000DAE631F6143F000800000020E000000080
:103F0000682E0008F43F0008E0000020B8440000DC
:103F1000782E0008000000000000000000000000F3
:103F20000000000000000000000000000000000091
:103F30000000000000000000000000000000000081
:103F40000000000000000000000000000000000071
:103F50000000000000000000000000000000000061
:103F60000000000000000000000000000000000051
:103F70000000000000000000000000000000000041
:103F8000ACF7FF1FE8F7FF1F107AFF1FACF7FF1F0A
:103F9000107AFF1F20F4F01F5000F81F5000F81F88
:103FA0009075FF1F20F4F01F0000000000000000CB
:103FB0000000000000000000000000000000000001
:103FC00001020304010203040607080902040608AB
:103FD00000366E0100000000000000000102030432
:103FE00006070809000000000000000000000000B3
:043FF00000000000CD
:0400000508000131BD
:00000001FF
